:020000040000FA
:1000000001288301850107309900831600309F0085
:10001000E830850083120B138501851D32280330DB
:10002000850000000000000000000000000000004B
:100030000630850000000000000000000000000005
:1000400000001430850000000000000000000000E7
:1000500000000000113085000000000000000000DA
:1000600000000F284F20A1204F20A1204F20A120C9
:100070007820CA204F20A1204F20A1204F20A1206E
:100080007820CA204F20A1204F20A1204F20A1205E
:100090007820D020D020D020D020D0203228A0011D
:1000A0001E30A100013085000000000000000000AB
:1000B0000000000000000000000000000000000040
:1000C000000000000000000000308500A00B69283F
:1000D0007528000000000000000000000000000083
:1000E00000000000000000005228A10B6D2808004D
:1000F000A0015A30A100013085000000000000007E
:1001000000000000000000000000000000000000EF
:100110000000000000000000000000308500A00B7F
:1001200092289E280000000000000000000000004F
:10013000000000000000000000007B28A10B9628B2
:100140000800A0011E30A100000000000000000017
:10015000000000000000000000000000000000009F
:10016000000000000000000000000000000000008F
:10017000A00BBB28C7280000000000000000000002
:10018000000000000000000000000000A428A10BF7
:10019000BF2808000330A200A120A20BCC28080031
:0C01A0000730A200A120A20BD22808000A
:02400E00C63FAB
:00000001FF
